:100000000C942A000C9447000C9447000C94470071
:100010000C9447000C9447000C9447000C94470044
:100020000C9447000C949E040C9447000C944700D9
:100030000C9447000C9434030C94D3020C944700A6
:100040000C9447000C9447000C9447000C94470014
:100050000C94470011241FBECFE5D8E0DEBFCDBF12
:1000600011E0A0E6B0E0E4E5F4E302C005900D92F3
:10007000AE32B107D9F712E0AEE2B1E001C01D9295
:10008000A138B107E1F70E9449000C94281A0C949A
:100090000000DF93CF930F92CDB7DEB71982109295
:1000A000B60101C000008091B601882F90E0823037
:1000B000910509F445C0833091053CF4009709F49B
:1000C000AAC08130910551F1BCC08430910549F03E
:1000D000843091050CF46BC08530910509F4B5C0EE
:1000E000B0C08BEB91E00E94BB0D89E991E00E94CA
:1000F000BB0D8091CB01853009F0A9C08091A90189
:10010000853009F0A6C01092CB011092A90181E0C0
:100110008093BA0181E08093B601A2C08091BB01B7
:10012000803521F48BEB91E00E94010C80919901C4
:10013000803509F090C089E991E00E94010C90C0DF
:100140008091D70181708823A9F48091B5018170D5
:10015000882381F480914601882361F087E491E04F
:1001600060E570E00E94D81289831092460181E018
:100170008093BA018091BB01803529F48BEB91E02B
:100180000E94591005C08091D7018E7F8093D701BE
:1001900080919901803529F489E991E00E945910F4
:1001A0005FC08091B5018E7F8093B50159C0809169
:1001B000BB01803521F48BEB91E00E941B088091FC
:1001C0009901803521F489E991E00E941B08809112
:1001D000A801893029F080919901803509F43DC04A
:1001E0008091CA01893021F08091BB018035B9F13D
:1001F00080919901803511F40E947E028091BB01AB
:10020000803511F40E946E0281E08093BA0181E092
:100210008093B60125C00E94CB0978948091990102
:10022000803521F48091BB01803521F084E08093FA
:10023000B60103C081E08093B60181E08093BA01EA
:100240000FC081E08093B6010BC0000009C0000020
:1002500007C0000005C0000003C0000001C000008E
:100260008091B601813041F08091B601823021F059
:100270008091B6018430D1F48BEB91E00E94200D87
:10028000882339F08BEB91E00E94C20F81E08093CC
:10029000BA0189E991E00E94200D882339F089E9AB
:1002A00091E00E94C20F81E08093BA018091BA016F
:1002B000882321F00E94320A1092BA018091D40161
:1002C0009091D501009739F58091D60180788823E7
:1002D000E1F08091D6018072882339F08091D701B6
:1002E000897F82608093D70106C08091D701897F82
:1002F00084608093D7012091CC013091CD018BEBAC
:1003000091E063E0F901099506C080E293E09093E3
:10031000D5018093D4018091B2019091B3010097EF
:1003200039F58091B40180788823E1F08091B4019F
:100330008072882339F08091B501897F8260809333
:10034000B50106C08091B501897F84608093B501B5
:100350002091AA013091AB0189E991E063E0F901B4
:10036000099506C080E293E09093B3018093B201B7
:100370000E94D20E9091B60180914301981709F422
:1003800091CE8091B601282F30E000D000D000D06F
:100390008DB79EB7019640E650E0FC015183408343
:1003A0004CE750E0FC0153834283FC0135832483F6
:1003B0000E9405178DB79EB706960FB6F8949EBF9C
:1003C0000FBE8DBF8091B601809343016CCEDF9349
:1003D000CF9300D00F92CDB7DEB79A8389836B831A
:1003E0008B81882F90E08230910559F183309105FF
:1003F00009F44AC08130910509F06AC088E390E0B1
:1004000028E330E0F901408129813A81F901248112
:100410002423FC01208389819A81FC01238D20689B
:10042000FC01238F89819A81FC01238D2062FC01CC
:10043000238F89819A81FC01238D2F7BFC01238FDF
:1004400047C088E390E028E330E0F901408129814A
:100450003A81F90125812423FC01208389819A8135
:10046000FC01238D2068FC01238F89819A81FC0186
:10047000238D2064FC01238F89819A81FC01238DC7
:100480002F7DFC01238F24C088E390E028E330E037
:10049000F901408129813A81F9012381242BFC0152
:1004A000208389819A81F1E089399F0711F40E94A4
:1004B0007E0289819A8121E08B3B920711F40E9490
:1004C0006E0289819A81FC01238D2F77FC01238F95
:1004D0000F900F900F90CF91DF910895DF93CF93FE
:1004E000CDB7DEB78BEB91E020E030E0B9014DE114
:1004F00050E00E943A19CF91DF910895DF93CF9396
:10050000CDB7DEB789E991E02DE130E0B9014DE1E9
:1005100050E00E943A19CF91DF910895DF93CF9375
:1005200000D00F92CDB7DEB789837B836A83809139
:100530005D0290915E0201969C012F773070809150
:100540005B0290915C0228173907E1F080915D020F
:1005500090915E0285529E4F2981FC0120838091FB
:100560005D0290915E02019690935E0280935D021F
:1005700080915D0290915E028F77907090935E0201
:1005800080935D028AE290E02AE230E0F901208166
:100590002062FC01208380E090E00F900F900F908C
:1005A000CF91DF9108951F920F920FB60F921124F1
:1005B0002F933F938F939F93EF93FF93DF93CF936B
:1005C000CDB7DEB720915D0230915E0280915B0273
:1005D00090915C022817390701F18CE290E020919C
:1005E0005B0230915C0225523E4FF9012081FC01F3
:1005F000208380915B0290915C02019690935C0253
:1006000080935B0280915B0290915C028F77907087
:1006100090935C0280935B0209C08AE290E02AE238
:1006200030E0F90120812F7DFC012083CF91DF9103
:10063000FF91EF919F918F913F912F910F900FBE5E
:100640000F901F901895DF93CF9300D00F92CDB7E6
:10065000DEB789837B836A8380E090E00F900F9000
:100660000F90CF91DF9108951F920F920FB60F92C6
:1006700011242F933F938F939F93EF93FF93DF93D7
:10068000CF93CDB7DEB72597DEBFCDBF8CE290E02C
:10069000FC0180818D8380913E01882F90E0813024
:1006A000910509F440C0823091051CF4009751F087
:1006B000A2C08230910509F490C08330910509F4FD
:1006C00060C099C087E491E09093B9018093B8012C
:1006D0001C821B820BC08B819C81895B9E4FFC011D
:1006E00010828B819C8101969C838B838B819C8162
:1006F0008035910580F38D818D3009F477C08D812F
:100700008A3009F475C08091B8019091B9012D81AA
:10071000FC01208301969093B9018093B80181E098
:1007200080933E0168C02091B8013091B90187E9FA
:1007300091E02817390708F05DC08D818D3019F0E0
:100740008D818A3089F48091B8019091B901F1E0EE
:1007500087349F0739F030F081E08093460183E0D1
:1007600080933E01000047C08091B8019091B9018B
:100770002D81FC01208301969093B9018093B801EB
:100780003AC080914601882321F587E491E0909357
:10079000B9018093B8011A8219820BC089819A81AC
:1007A000895B9E4FFC01108289819A8101969A8310
:1007B000898389819A818035910580F38091B80180
:1007C0009091B9012D81FC01208381E080933E014D
:1007D00012C082E080933E010EC08D818D3019F0F1
:1007E0008D818A3041F410923E0105C0000003C0A3
:1007F000000001C000002596DEBFCDBFCF91DF9184
:10080000FF91EF919F918F913F912F910F900FBE8C
:100810000F901F901895DF93CF93CDB7DEB787E386
:1008200090E02FE1FC01208388E390E028E330E0B2
:10083000F90120812160FC01208388E390E028E316
:1008400030E0F90120812260FC01208388E390E000
:1008500028E330E0F90120812460FC01208388E353
:1008600090E028E330E0F90120812860FC0120833A
:1008700088E390E028E330E0F90120812061FC0169
:10088000208382E390E022E330E0F90120812064BC
:10089000FC01208382E390E022E330E0F901208133
:1008A0002068FC0120838AE390E0FC0110828BE346
:1008B00090E02BE330E0F90120812160FC012083EE
:1008C0008BE390E02BE330E0F90120812260FC0112
:1008D00020838BE390E02BE330E0F901208124605A
:1008E000FC0120838BE390E02BE330E0F9012081D1
:1008F0002860FC0120838BE390E02BE330E0F901DA
:1009000020812061FC012083CF91DF910895DF9346
:10091000CF93CDB7DEB78FE490E0FC0110828EE478
:1009200090E023E0FC0120838CE490E02EE83DEF92
:10093000FC0131832083CF91DF9108951F920F92A4
:100940000FB60F9211242F933F938F939F93EF93A2
:10095000FF93DF93CF93CDB7DEB788E390E028E332
:1009600030E0F90120812061FC0120838CE490E0DB
:100970002EE83DEFFC013183208380913F0190916F
:100980004001009749F080913F019091400101970B
:100990009093400180933F018091D4019091D501C3
:1009A000009749F08091D4019091D50101979093DF
:1009B000D5018093D4018091B2019091B301009749
:1009C00049F08091B2019091B30101979093B301E6
:1009D0008093B2018091970190919801009749F01E
:1009E000809197019091980101979093980180933D
:1009F00097018091D9019091DA01009749F0809197
:100A0000D9019091DA0101979093DA018093D9018D
:100A10008091410190914201009749F080914101FC
:100A200090914201019790934201809341018091FE
:100A3000440190914501009749F0809144019091C3
:100A40004501019790934501809344018091C8012D
:100A50009091C901009749F08091C8019091C90116
:100A600001979093C9018093C8018091A60190914C
:100A7000A701009749F08091A6019091A7010197E5
:100A80009093A7018093A60189E390E0FC01808107
:100A9000882F90E0817090700097E9F410922F01F8
:100AA00080915F028170882371F580912E018F5FA4
:100AB00080932E0180912E01833038F110922E0107
:100AC00080915F02816080935F0280915F028D7FE1
:100AD00080935F021BC010922E0180915F02817093
:100AE0008823A1F080912F018F5F80932F01809147
:100AF0002F01833058F080915F028E7F80935F02D8
:100B000010922F0103C0000001C0000089E390E0B3
:100B1000FC018081882F90E0827090700097E9F44A
:100B20001092310180915F028270882371F580916B
:100B300030018F5F8093300180913001833038F134
:100B40001092300180915F02826080935F028091F9
:100B50005F028E7F80935F021BC0109230018091F4
:100B60005F0282708823A1F0809131018F5F8093B2
:100B7000310180913101833058F010923101809120
:100B80005F028D7F80935F0203C0000001C0000000
:100B900089E390E0FC018081882F90E08470907060
:100BA0000097E9F41092330180915F0284708823EA
:100BB00061F5809132018F5F809332018091320123
:100BC000833028F11092320180915F02846080931B
:100BD0005F0280915F02877F80935F0219C010924D
:100BE000320180915F028470882391F080913301FB
:100BF0008F5F8093330180913301833048F080917F
:100C00005F028B7F80935F0203C0000001C0000081
:100C100089E390E0FC018081882F90E088709070DB
:100C20000097E9F41092350180915F028870882363
:100C300071F5809134018F5F80933401809134018C
:100C4000833038F11092340180915F028860809384
:100C50005F0280915F028B7F80935F021BC01092C6
:100C6000340180915F0288708823A1F08091350162
:100C70008F5F8093350180913501833058F0109259
:100C8000330180915F02877F80935F0203C0000081
:100C900001C0000080E390E0FC018081882F90E09B
:100CA000807490700097E9F41092390180915F028E
:100CB0008071882371F5809138018F5F80933801AE
:100CC00080913801833038F11092380180915F02B1
:100CD000806180935F028091D60180618093D6010C
:100CE0001BC01092380180915F0280718823A1F0AF
:100CF000809139018F5F8093390180913901833070
:100D000058F01092390180915F028F7E80935F02CC
:100D100003C0000001C0000080E390E0FC0180817E
:100D20008823ECF01092370180915F028072882353
:100D300071F5809136018F5F809336018091360185
:100D4000833038F11092360180915F028062809387
:100D50005F028091B40180618093B4011BC0109246
:100D6000360180915F0280728823A1F08091370163
:100D70008F5F8093370180913701833058F0109254
:100D8000370180915F028F7D80935F0203C0000076
:100D900001C0000089E390E0FC018081882F90E091
:100DA000807190700097C1F410923B0180915F02B6
:100DB0008074882349F580913A018F5F80933A01CE
:100DC00080913A01833010F110923A0180915F02D4
:100DD000806480935F021BC010923A0180915F0291
:100DE00080748823A1F080913B018F5F80933B0149
:100DF00080913B01833058F010923B0180915F025B
:100E00008F7B80935F0203C0000001C0000089E374
:100E100090E0FC018081882F90E0807290700097B4
:100E2000C1F410923D0180915F028078882349F5DA
:100E300080913C018F5F80933C0180913C01833025
:100E400010F110923C0180915F02806880935F02F4
:100E50001BC010923C0180915F0280788823A1F032
:100E600080913D018F5F80933D0180913D018330F2
:100E700058F080915F028F7780935F0210923D015E
:100E800003C0000001C00000CF91DF91FF91EF91FE
:100E90009F918F913F912F910F900FBE0F901F90B8
:100EA0001895DF93CF93CDB7DEB780E490E0FC01D7
:100EB000108289E290E023E3FC0120838AE290E043
:100EC0002AE230E0F90120812861FC01208387E4D7
:100ED00091E09093B9018093B8018AE290E02AE210
:100EE00030E0F90120812068FC012083CF91DF915F
:100EF0000895DF93CF9300D00F92CDB7DEB78B83E9
:100F00008B81807F8A838A8182958F708A838A8190
:100F1000805D8A838A818A3318F08A81895F8A8317
:100F20008B818F70805D898389818A3318F08981F4
:100F3000895F89838A81882F90E0209160003091B9
:100F40006100B9010E948E028981882F90E0209172
:100F5000600030916100B9010E948E020F900F90E5
:100F60000F90CF91DF910895DF93CF93CDB7DEB788
:100F700060970FB6F894DEBF0FBECDBF6D877E873A
:100F80008F87988B19861A861B861C863DC01D820A
:100F90001E821F82188624C019821A821B821C821C
:100FA0000BC089819A81AB81BC810196A11DB11DC5
:100FB00089839A83AB83BC8389819A81AB81BC810D
:100FC000803B9105A105B10560F38D819E81AF81C4
:100FD000B8850196A11DB11D8D839E83AF83B8870F
:100FE0008D819E81AF81B88588329105A105B105BB
:100FF00098F289859A85AB85BC850196A11DB11DA6
:1010000089879A87AB87BC8729853A854B855C851C
:101010008D859E85AF85B889281739074A075B07F4
:1010200008F4B5CF60960FB6F894DEBF0FBECDBF03
:10103000CF91DF910895DF93CF9300D0CDB7DEB786
:101040009A83898389819A81FC018785882F90E022
:101050008530910509F4BFC08630910594F4813044
:101060009105F9F08230910524F4009709F460C1EC
:1010700071C18330910519F18430910509F400C1E3
:1010800069C18730910509F4A0C087309105CCF182
:101090008830910509F46DC08930910509F471C15A
:1010A00059C189819A81FC0185859685009709F04F
:1010B0006AC189819A8123E0FC01278767C1898100
:1010C0009A8120E233E0FC01328F218F89819A815D
:1010D000FC01248D297FFC01248F89819A81FC01E8
:1010E000168289819A81FC012189328989819A81BC
:1010F00062E0F901099589819A8126E0FC01278740
:1011000045C189819A81FC01838D8071882371F0AA
:1011100089819A8120E233E0FC01328F218F89811D
:101120009A81FC01238D2F7EFC01238F89819A8176
:10113000FC01848D86708430B1F489819A81FC0130
:101140002189328989819A8163E0F9010995898130
:101150009A81FC01248D297FFC01248F89819A8149
:1011600028E0FC01278789819A81FC01148A138A6F
:101170000DC189819A81FC01168289819A81FC01C5
:101180001286118689819A81FC01148A138A8981C9
:101190009A81FC01248D297FFC01248F89819A8109
:1011A00020E233E0FC01328F218F89819A81FC019A
:1011B0002189328989819A8161E0F90109958981C2
:1011C0009A8127E0FC012787E1C089819A8125E087
:1011D000FC012787DBC089819A81FC01838D8071A6
:1011E000882379F189819A81FC018681282F2F5FDC
:1011F00089819A81FC01268389819A81FC018681FB
:10120000823071F489819A81FC01818D928D20E276
:1012100033E0281B390B89819A81FC0130872783B1
:1012200081E08093BA0189819A81FC01238D2F7E10
:10123000FC01238F89819A8120E233E0FC01328F07
:10124000218F89819A81FC01848D8670823009F01A
:101250009CC089819A81FC012189328989819A8186
:1012600063E0F901099589819A8124E0FC012787CF
:1012700089819A81FC01248D297FFC01248F86C0FD
:1012800089819A81FC01268189819A81FC012283CE
:1012900089819A8128E631E0FC01348B238B898196
:1012A0009A81FC018281282F30E088E691E0B90123
:1012B0000E94C516CB01282F2F7089819A812F702B
:1012C000FC01338D307F232BFC01238F89819A8190
:1012D000FC018781908529813A81F901238D2F7046
:1012E000222F30E0B9010E94B116CB019C01898107
:1012F0009A81FC013287218789819A81FC01248DA2
:10130000297FFC01248F89819A8123E4FC01278BAA
:1013100089819A81FC01248D297FFC01248F898198
:101320009A8129E0FC01278781E08093BA012EC0D1
:1013300089819A8124E630E0FC01368725878981FE
:101340009A8121E0FC01278789819A8120E2FC01B2
:10135000278B1CC089819A81FC012189328989816E
:101360009A8163E0F901099589819A8124E630E048
:10137000FC013687258789819A8121E0FC01278736
:1013800005C0000003C0000001C000000F900F90D6
:10139000CF91DF910895DF93CF93CDB7DEB70E9451
:1013A0000B040E9451078DE00E9459160E94A0155F
:1013B0000E9487048BEB91E020E030E0B9014DE121
:1013C00050E00E942A1989E991E02DE130E0B9014D
:1013D0004DE150E00E942A1983E08093BE018EEF18
:1013E0008093BF018DEF8093C0018CE080939C01BE
:1013F0008BEF80939D0187EF80939E0180E293E0C5
:101400009093D5018093D40180E293E09093B3014F
:101410008093B2018091D70181608093D701809140
:10142000B50181608093B501109246011092CA0106
:101430001092CB011092A8011092A90187EE91E0C1
:101440009093CD018093CC0187EE91E09093AB0116
:101450008093AA0189E590E024E0FC012083CF91EC
:10146000DF910895DF93CF9300D0CDB7DEB780E052
:1014700060E00E947D158091B601882F90E0823057
:10148000910509F4F4C08330910544F4009709F400
:10149000BCC08130910509F443C0AEC184309105D0
:1014A00009F46CC1843091050CF0A5C182E890E08C
:1014B0002EE630E061E070E040E150E00E94191754
:1014C0008091C101482F50E080919F01282F30E08A
:1014D0008DB79EB708970FB6F8949EBF0FBE8DBF0D
:1014E0008DB79EB701966EE670E0DC016D937C933C
:1014F00063E970E0FC0173836283DC0115965C9301
:101500004E931497FC01378326830E9405178DB7ED
:101510009EB708960FB6F8949EBF0FBE8DBF6CC1E4
:10152000A091CE01B091CF01BA83A9836091AC01A3
:101530007091AD018091D201482F50E08091B001AF
:10154000282F30E0EDB7FEB73C970FB6F894FEBFFA
:101550000FBEEDBF8DB79EB70196AEE6B0E0FC01C1
:10156000B183A083A8EAB0E0FC01B383A283E98140
:10157000FA81DC011596FC93EE931497DC01179623
:101580007C936E931697FC0151874087DC011B9674
:101590003C932E931A970E940517EDB7FEB73C9621
:1015A0000FB6F894FEBF0FBEEDBF8091C101482F6A
:1015B00050E080919F01282F30E08DB79EB70897AB
:1015C0000FB6F8949EBF0FBE8DBF8DB79EB7019624
:1015D0006EE670E0DC016D937C936DEB70E0FC01D6
:1015E00073836283DC0115965C934E931497FC0120
:1015F000378326830E9405178DB79EB708960FB6CE
:10160000F8949EBF0FBE8DBFF7C08091C101482FD7
:1016100050E080919F01282F30E0ADB7BEB71897FA
:101620000FB6F894BEBF0FBEADBF8DB79EB7019683
:101630006EE670E0FC017183608362ED70E0DC01B6
:1016400013967C936E931297FC0155834483DC01BF
:1016500017963C932E9316970E940517EDB7FEB789
:1016600038960FB6F894FEBF0FBEEDBFC5C080918F
:10167000CE019091CF019A8389836091AC017091E2
:10168000AD018091D201482F50E08091B001282F08
:1016900030E0ADB7BEB71C970FB6F894BEBF0FBE13
:1016A000ADBF8DB79EB70196AEE6B0E0FC01B18349
:1016B000A083A8EAB0E0FC01B383A283E981FA81A8
:1016C000DC011596FC93EE931497DC0117967C933E
:1016D0006E931697FC0151874087DC011B963C9363
:1016E0002E931A970E940517EDB7FEB73C960FB6DA
:1016F000F894FEBF0FBEEDBF80E061E00E947D1553
:1017000080917602882319F427EE30E002C026E7A4
:1017100032E06091D0017091D1014091AE015091C1
:10172000AF018DB79EB70A970FB6F8949EBF0FBE54
:101730008DBF8DB79EB70196EEE6F0E0DC01ED932C
:10174000FC93ECEEF0E0DC011396FC93EE93129721
:10175000FC0135832483DC0117967C936E931697E6
:10176000FC01518740870E9405178DB79EB70A96E6
:101770000FB6F8949EBF0FBE8DBF3EC08AEF90E0BB
:101780002EE630E061E070E040E150E00E94191781
:101790008091BB01803559F48BE091E02EE630E07A
:1017A00061E070E048E050E00E9419170AC084E14F
:1017B00091E02EE630E061E070E047E050E00E940A
:1017C000191780919901803559F48CE191E02EE64A
:1017D00030E061E070E048E050E00E9419170CC072
:1017E00085E291E02EE630E061E070E047E050E015
:1017F0000E94191701C000000F900F90CF91DF9148
:101800000895DF93CF9300D0CDB7DEB79A83898355
:1018100089819A81FC01848D8670882309F44BC0EC
:1018200089819A81FC01848D8670843029F48981B4
:101830009A81FC01168214C089819A81FC018789F2
:10184000882349F089819A81FC01228189819A81CA
:10185000FC01268305C089819A8124E2FC0126834C
:1018600089819A81FC01108E89819A81FC0186818F
:10187000282F30E089819A81FC01838D8F70882F19
:1018800090E0A901489F9001499F300D589F300D6D
:10189000112489819A81FC01348B238B89819A815F
:1018A000FC012189328989819A8163E0F9010995D6
:1018B00081E08093BA0180915F028170882309F1F1
:1018C0008091D6018078882309F04EC08091D7019D
:1018D0008670823009F44AC08091D701897F809355
:1018E000D70180E293E09093D5018093D4012091B9
:1018F000CC013091CD018BEB91E061E0F9010995CC
:101900003AC080915F0282708823F9F08091D601FD
:101910008078882369F58091D7018670843051F1F1
:101920008091D701897F8093D70180E293E09093E3
:10193000D5018093D4012091CC013091CD018BEB66
:1019400091E062E0F901099516C08091D601807896
:10195000882389F02091CC013091CD018BEB91E06F
:1019600063E0F901099507C0000005C0000003C04D
:10197000000001C0000080915F028470882309F19B
:101980008091B4018078882309F04EC08091B50120
:101990008670823009F44AC08091B501897F8093B6
:1019A000B50180E293E09093B3018093B20120915E
:1019B000AA013091AB0189E991E061E0F901099553
:1019C0003AC080915F0288708823F9F08091B40159
:1019D0008078882369F58091B5018670843051F153
:1019E0008091B501897F8093B50180E293E0909367
:1019F000B3018093B2012091AA013091AB0189E932
:101A000091E062E0F901099516C08091B4018078F7
:101A1000882389F02091AA013091AB0189E991E0F6
:101A200063E0F901099507C0000005C0000003C08C
:101A3000000001C000000F900F90CF91DF9108953A
:101A4000DF93CF9300D000D00F92CDB7DEB79D8348
:101A50008C8319828C819D81FC01838D8071882308
:101A6000E9F18C819D81FC01838D8072882351F086
:101A70008C819D81FC018681282F2F5F8C819D8127
:101A8000FC0126838C819D81FC01838D80748823D9
:101A900081F08C819D81FC018681882351F08C81AD
:101AA0009D81FC018681282F21508C819D81FC0124
:101AB00026838C819D81FC01108E81E089838C813D
:101AC0009D81FC01238D2F7EFC01238F8C819D81C4
:101AD00020E233E0FC01328F218F44C08C819D8154
:101AE000FC01838D80788823E9F18C819D81FC0144
:101AF000818D928D20E233E0281B390B8C819D81F2
:101B0000FC01348723878C819D81FC0123853485EA
:101B10008C819D81FC01818592852817390710F100
:101B20008C819D81FC01838594852C813D81F90107
:101B300021853285B9010E94B116CB019B838A832E
:101B40008C819D81FC01808D282F30E08A819B81D2
:101B50002817390739F02A818C819D81FC01208F5B
:101B600081E0898389810F900F900F900F900F90E3
:101B7000CF91DF910895DF93CF9300D0CDB7DEB73B
:101B80009A83898389819A81FC018089882F90E0DA
:101B90008230910509F48DC08330910534F40097AB
:101BA00089F08130910529F1F8C08430910509F45C
:101BB000CBC0843091050CF464C08530910509F4E4
:101BC000D6C0EBC089819A8120E233E0FC01328FDC
:101BD000218F89819A81FC012189328989819A81A9
:101BE00061E0F901099589819A8121E0FC01208B4E
:101BF000D4C089819A81FC01838D80718823D9F0BA
:101C000089819A81FC012189328989819A8163E0E5
:101C1000F901099589819A8120E5FC01208384EFEF
:101C200091E0909345018093440189819A8124E059
:101C3000FC01208BB2C089819A81FC01848D867061
:101C4000823009F0A3C089819A81FC01248D297F0B
:101C5000FC01248F89819A81FC0121893289898143
:101C60009A8163E0F901099589819A8128EC30E035
:101C7000FC013687258789819A8123E0FC01208B2E
:101C80008CC089819A81FC0185859685009709F031
:101C90007FC089819A81FC012189328989819A8159
:101CA00062E0F901099589819A8122E0FC01208B8B
:101CB00074C089819A81FC01838D80718823D9F059
:101CC00089819A81FC012189328989819A8163E025
:101CD000F901099589819A8120E5FC01208384EF2F
:101CE00091E0909345018093440189819A8124E099
:101CF000FC01208B52C089819A81FC01848D867001
:101D0000843009F047C089819A81FC01248D297FA4
:101D1000FC01248F89819A81FC0121893289898182
:101D20009A8163E0F901099589819A81FC01108209
:101D300084EF91E0909345018093440189819A81D9
:101D400024E0FC01208B29C0809144019091450141
:101D5000009711F589819A81FC01248D297FFC016E
:101D6000248F89819A8125E0FC01208B16C089810E
:101D70009A81FC01248D297FFC01248F89819A811D
:101D800020E233E0FC01328F218F07C0000005C044
:101D9000000003C0000001C000000F900F90CF9121
:101DA000DF910895DF93CF93CDB7DEB78091B60171
:101DB000882F90E08230910509F45CC08330910552
:101DC0003CF4009709F4D4C08130910531F0D7C0BC
:101DD0008330910509F495C0D2C080915F02807470
:101DE0008823E9F01092CA011092A80183E0809341
:101DF000B60181E08093BA012091CC013091CD01F0
:101E00008BEB91E063E0F90109952091AA013091F3
:101E1000AB0189E991E063E0F9010995B0C08091D7
:101E20005F028078882309F4A5C082E08093B60120
:101E30002091CC013091CD018BEB91E063E0F90171
:101E400009952091AA013091AB0189E991E063E005
:101E5000F90109958091D70181608093D701809124
:101E6000B50181608093B50181E08093BA01109241
:101E7000460185C080915F028170882381F4809142
:101E80005F028270882359F480915F0284708823F6
:101E900031F480915F028870882309F46DC08091CD
:101EA000D701897F8093D7018091B501897F809385
:101EB000B5012091CC013091CD018BEB91E063E035
:101EC000F90109952091AA013091AB0189E991E0CE
:101ED00063E0F90109958091D70181608093D70172
:101EE0008091B50181608093B50181E08093BA0152
:101EF00080915F028F7780935F0281E08093B601CB
:101F00003EC080915F028170882379F480915F02E6
:101F10008270882351F480915F028470882329F4B1
:101F200080915F028870882349F18091D701897F71
:101F30008093D7018091B501897F8093B50120916D
:101F4000CC013091CD018BEB91E063E0F901099573
:101F50002091AA013091AB0189E991E063E0F90198
:101F6000099581E08093B60181E08093BA0107C0B2
:101F7000000005C0000003C0000001C00000CF91B8
:101F8000DF910895DF93CF9300D0CDB7DEB79A836A
:101F9000898389819A81FC01838D8072882319F15C
:101FA00089819A81FC018681282F30E089819A817C
:101FB000FC01838D8F70882F90E0A901489F9001CC
:101FC000499F300D589F300D112489819A81FC0161
:101FD000808D882F90E0280F391F89819A81FC011C
:101FE000348B238B3DC089819A81FC0186818823B3
:101FF00019F189819A81FC018681282F30E089813D
:102000009A81FC01838D8F70882F90E0A901489FF1
:102010009001499F300D589F300D112489819A817C
:10202000FC01808D882F90E0281B390B89819A81D3
:10203000FC01348B238B14C089819A81FC01838D30
:102040008F70282F30E089819A81FC01808D882F44
:1020500090E0281B390B89819A81FC01348B238BFA
:1020600089819A81FC018389948999234CF489811F
:102070009A81FC01148A138A89819A81FC01108E4D
:1020800089819A81FC0183899489F1E089369F07CF
:102090005CF089819A8128E631E0FC01348B238B46
:1020A00089819A81FC01108E0F900F90CF91DF9162
:1020B0000895DF93CF9300D000D00F92CDB7DEB755
:1020C0009D838C838C819D81FC01858596850097FD
:1020D00009F032C11B828C819D81FC01848D81704D
:1020E000882319F18C819D81FC01238934898C819D
:1020F0009D81FC01368B258B8C819D81FC01248D7B
:102100002E7FFC01248F8C819D81FC01248D297FF1
:10211000FC01248F82E080933E011092760210929F
:10212000460181E08093BA0108C18C819D81FC0148
:10213000238934898C819D81FC0185899689A90137
:10214000481B590BCA019A8389838C819D81FC01AC
:10215000838D8078882339F089819A8190937502E4
:102160008093740216C089819A818530910534F478
:1021700089819A81FFEF8C3F9F073CF489819A8186
:10218000909375028093740204C0109275021092AD
:1021900074028091740290917502181619060CF061
:1021A00042C08C819D81FC01838D8078882309F554
:1021B0008C819D81FC01848D86708430D1F08C816E
:1021C0009D8120E233E0FC01328F218F8C819D8143
:1021D000FC01248D297FFC01248F8C819D81FC01D1
:1021E000218932898C819D8162E0F9010995000085
:1021F0007AC08C819D81FC01838D8072882309F4D3
:102200006FC08C819D81FC01218932898C819D81E7
:1022100063E0F90109958C819D8120E931E0FC01A1
:102220003687258760C0809174029091750299234A
:102230000CF041C08C819D81FC01838D80788823C6
:1022400009F58C819D81FC01848D86708230D1F0EE
:102250008C819D8120E233E0FC01328F218F8C81C3
:102260009D81FC01248D297FFC01248F8C819D811F
:10227000FC01218932898C819D8161E0F9010995F8
:10228000000031C08C819D81FC01838D8074882386
:1022900049F18C819D81FC01218932898C819D814C
:1022A00063E0F90109958C819D8120E931E0FC0111
:1022B0003687258718C08C819D81FC01838D8078AD
:1022C000882389F08C819D81FC01218932898C8150
:1022D0009D8163E0F901099581E08093BA0103C013
:1022E000000001C000008C819D81FC01848D8670FE
:1022F000882319F18C819D81FC01838D807888234E
:10230000E1F08C819D81FC01218932898C819D8144
:1023100063E0F901099581E08093BA018C819D8188
:1023200020E233E0FC01328F218F81E08093BA01FB
:1023300081E08093B60101C000000F900F900F90D4
:102340000F900F90CF91DF910895DF93CF93CDB78A
:10235000DEB761970FB6F894DEBF0FBECDBF198A06
:10236000188A1F861E861D861C861D821B861A865D
:102370004AC08A859B85895B9E4FFC0180818134A0
:10238000E9F58A859B850196895B9E4FFC018081DA
:102390008A35A1F58A859B8502969F838E8319864F
:1023A000188616C08885998528853985295B3E4F12
:1023B000F90120818A589D4FFC01208388859985E9
:1023C0008830910581F0888599850196998788875D
:1023D0008A859B859C01215030408885998582178C
:1023E000930704F301C00000888599858A589D4FA2
:1023F000FC01108281E090E09D878C878A859B8517
:1024000001969B878A878A859B85803591050CF488
:10241000B0CF8C859D85009791F11986188615C0DF
:10242000888599854E815F8128853985240F351FE0
:10243000295B3E4FF901208186599D4FFC01208385
:10244000888599850196998788872E813F8188851F
:102450009985820F931F895B9E4FFC018081882F95
:1024600090E0C0978A309105D8F288859985865981
:102470009D4FFC01108281E090E0998B888B2E812A
:102480003F8188859985820F931F9B878A874AC0E1
:102490008A859B85895B9E4FFC0180818534C9F5C7
:1024A0008A859B850196895B9E4FFC0180818C34D7
:1024B00081F5198618868A859B8502969B878A876F
:1024C00016C0888599852A853B85295B3E4FF90191
:1024D0002081805A9D4FFC01208388859985019633
:1024E000998788878A859B8501969B878A878A85B5
:1024F0009B85895B9E4FFC018081882F90E0C0976F
:102500008A309105F0F288859985805A9D4FFC01AB
:10251000108281E090E09F878E878A859B85019657
:102520009B878A878A859B85803591050CF4B0CF7F
:1025300088899989009791F18E859F85009771F11F
:102540008AE692E00E94D8169C838B8380E692E014
:102550000E94D8169A8389838B819C819923F4F0F9
:102560008B819C81F1E089369F07C4F489819A812F
:102570009923A4F089819A8121E08936920774F425
:102580008B819C819093D1018093D00189819A8124
:102590009093AF018093AE0181E08D838D81619630
:1025A0000FB6F894DEBF0FBECDBFCF91DF91089577
:1025B000DF93CF93CDB7DEB767970FB6F894DEBF42
:1025C0000FBECDBF9D8B8C8B7F8B6E8B8C899D8935
:1025D0009B8B8A8B8C899D89998B888B1B861A860D
:1025E000198618861F821E821D823FC0888999899C
:1025F000FC0180818134A1F5888999890196FC01CB
:1026000080818A3569F58889998901979C018C892F
:102610009D89A901481B590BCA018930910530F4E5
:102620008889998901979B8B8A8B05C08C899D89A4
:1026300008969B8B8A8B8A899B89FC01108286E78E
:1026400092E02C893D89B9010E94F61681E090E064
:102650009F838E83888999890296998B888B11C074
:10266000888999890196998B888B8E899F892C8975
:102670003D89280F391F888999898217930708F4A3
:10268000B5CF8E819F810097A9F1888999899D870F
:102690008C8781E090E09B878A8719C08E899F890B
:1026A00001972C893D89280F391F8C859D858217BC
:1026B000930750F4888999899C012D5F3F4F8C8541
:1026C0009D852817390718F41B861A8613C08C8538
:1026D0009D85FC018081882F90E0C09720E08A30A2
:1026E000910508F421E08C859D8501969D878C8756
:1026F0002223A1F68A859B85009709F47BC08C85EF
:102700009D85FC0110828AE692E028893989B90109
:102710000E94F6168C859D8501969D878C878C85F9
:102720009D859F878E875AC08E859F85FC018081FD
:10273000853409F04EC08E859F850196FC0180810D
:102740008C3409F046C08E859F8502969F878E87C0
:1027500081E090E0998788878E859F859D878C870B
:1027600019C08E899F8901972C893D89280F391FAF
:102770008C859D858217930750F48E859F859C01DB
:102780002D5F3F4F8C859D852817390718F41986D2
:10279000188613C08C859D85FC018081882F90E070
:1027A000C09720E08A30910508F421E08C859D8552
:1027B00001969D878C872223A1F68C859D85FC013F
:1027C000108280E692E02E853F85B9010E94F616C0
:1027D00011C08E859F8501969F878E878E899F89E0
:1027E0002C893D89280F391F8E859F858217930775
:1027F00008F49ACF8A859B85009791F18885998501
:10280000009771F18AE692E00E94D8169C838B8330
:1028100080E692E00E94D8169A8389838B819C81FE
:102820009923F4F08B819C81F1E089369F07C4F4F1
:1028300089819A819923A4F089819A8121E089363E
:10284000920774F48B819C819093D1018093D00185
:1028500089819A819093AF018093AE0181E08D834D
:102860008D8167960FB6F894DEBF0FBECDBFCF91B6
:10287000DF910895DF93CF9300D0CDB7DEB79A8371
:10288000898389819A81009711F400C006C08981EB
:102890009A810197F1F79A8389830F900F90CF91D6
:1028A000DF910895DF93CF93CDB7DEB785E390E056
:1028B00025E330E0F90120812064FC01208300C081
:1028C00085E390E025E330E0F90120812F7BFC01D6
:1028D0002083CF91DF910895DF93CF9300D00F92A3
:1028E000CDB7DEB78A836B838B81882351F085E374
:1028F00090E025E330E0F90120812061FC01208394
:1029000009C085E390E025E330E0F90120812F7EC6
:10291000FC01208385E390E025E330E0F90120818C
:102920002F7DFC01208384E390E024E330E0F90173
:1029300020812F60FC01208385E390E0FC018081F1
:10294000807F898385E390E02A81322F32953F7022
:102950002981232BFC0120830E94521485E390E0FF
:102960002A81322F3F702981232BFC0120830E9472
:10297000521485E390E029812F60FC0120830F90A1
:102980000F900F90CF91DF910895DF93CF9300D0F8
:10299000CDB7DEB78A838A81882351F085E390E042
:1029A00025E330E0F90120812061FC01208309C08A
:1029B00085E390E025E330E0F90120812F7EFC01E2
:1029C000208385E390E025E330E0F9012081206257
:1029D000FC01208384E390E024E330E0F9012081CE
:1029E000207FFC01208385E390E025E330E0F901BE
:1029F00020812064FC01208300C083E390E0FC017F
:102A000080818295807F898385E390E025E330E0B3
:102A1000F90120812F7BFC01208300C085E390E039
:102A200025E330E0F90120812064FC01208300C00F
:102A300083E390E0FC018081982F9F708981892B2E
:102A4000898385E390E025E330E0F90120812F7B45
:102A5000FC01208389810F900F90CF91DF91089521
:102A60001F93DF93CF93CDB7DEB780E00E94C514EC
:102A7000182F812F8823CCF384E090E00E943A1431
:102A800080E00E94C514CF91DF911F9108951F939C
:102A9000DF93CF930F92CDB7DEB7898389818034DE
:102AA00010F410E401C010E0812F80580E945D15E1
:102AB0000F90CF91DF911F910895DF93CF930F92E5
:102AC000CDB7DEB789830E943015898160E00E940E
:102AD0006C140F90CF91DF910895DF93CF930F92F5
:102AE000CDB7DEB789830E943015898161E00E94ED
:102AF0006C140F90CF91DF910895DF93CF9300D0A6
:102B0000CDB7DEB789836A838A81882329F48981D6
:102B100080580E945D1504C0898180540E945D1513
:102B20000F900F90CF91DF910895DF93CF93CDB7A2
:102B3000DEB70E943015882F90E0CF91DF91089585
:102B4000DF93CF93CDB7DEB781E00E945D15CF91C3
:102B5000DF910895DF93CF93CDB7DEB782E00E9477
:102B60005D15CF91DF910895DF93CF9300D000D012
:102B70000F92CDB7DEB78B837D836C830E943015B7
:102B80008A838B818A3021F48A810E94471536C05E
:102B90008B818830F1F48A81882319F48FE489834A
:102BA00009C08A81803419F48FE0898303C08A8147
:102BB000815089838981805860E00E946C1480E292
:102BC00061E00E946C148981805860E00E946C145E
:102BD00015C08A81803129F480EC60E00E946C1479
:102BE00007C08A81803521F480E860E00E946C147F
:102BF0000E9430158B8161E00E946C1480E090E0AF
:102C00000F900F900F900F900F90CF91DF9108953C
:102C10001F93DF93CF9300D0CDB7DEB79A8389831C
:102C200006C02EE630E0812FB9010E94B4158981DB
:102C30009A81FC011081812F882309F081E0282FDF
:102C400089819A8101969A838983222351F70F9073
:102C50000F90CF91DF911F9108951F93DF93CF9332
:102C600000D000D00F92CDB7DEB79D838C8306C015
:102C70002EE630E0812FB9010E94B4158C819D8130
:102C80009B838A838C819D8101969D838C838A811D
:102C90009B81FC01849189838981182F112341F73D
:102CA0000F900F900F900F900F90CF91DF911F9189
:102CB0000895DF93CF930F92CDB7DEB7898384E376
:102CC00090E024E330E0F90120812F67FC012083AC
:102CD00080E09DE70E943A1485E390E025E330E030
:102CE000F90120812260FC01208385E390E025E347
:102CF00030E0F90120812160FC0120830E94521400
:102D000080E097E20E943A140E94521480E890E01A
:102D10000E943A140E94521480E890E00E943A14F3
:102D200085E390E025E330E0F90120812E7FFC016E
:102D300020830E94521480E890E00E943A1488E2B6
:102D40000E945D1588E00E945D150E94A01586E036
:102D50000E945D1589810E945D150F90CF91DF91D2
:102D60000895AA1BBB1B51E107C0AA1FBB1FA617D2
:102D7000B70710F0A61BB70B881F991F5A95A9F724
:102D800080959095BC01CD01089597FB092E0726EB
:102D90000AD077FD04D0E5DF06D000201AF4709544
:102DA00061957F4F0895F6F7909581959F4F08950F
:102DB000FC0188279927E89421912032E9F32930F2
:102DC00010F02E30C8F32B3241F02D3239F46894D4
:102DD00004C00E94FD16820F911D219120532A30BC
:102DE000C0F31EF4909581959F4F0895FB01DC017F
:102DF00001900D920020E1F708957AE0979F902DC1
:102E0000879F802D910D11240895A0E0B0E0EBE0A4
:102E1000F7E10C94011A9E01275F3F4F8D819E813F
:102E20006F817885A9010E9452172096E2E00C94E8
:102E30001D1AA0E0B0E0EFE1F7E10C94F719EB0107
:102E40008A015901D90113962C91139721FF22C0B1
:102E5000C82ED92EEE24FF2417C0D5011896ED9167
:102E6000FC911997D6018C91B50109950097A1F4B1
:102E70000894C11CD11C0894811C911C8C169D06C1
:102E800060F30894E11CF11CE016F10628F4882494
:102E90009924F4CFEE24FF24C701CDB7DEB7ECE0D0
:102EA0000C94131AACE0B0E0E8E5F7E10C94F219E9
:102EB0006C012B018A01FC0117821682838181FD3E
:102EC00003C02FEF3FEFC1C14E010894811C911C3C
:102ED0006FE3362EF6019381F20193FD859193FF06
:102EE00081912F01882309F4ADC1853239F493FD16
:102EF000859193FF81912F01853229F490E0B601ED
:102F00000E946719E7CFEE24FF2420E02032B0F4BE
:102F10008B3269F08C3228F4803251F0833271F4B4
:102F20000BC08D3239F0803349F421602CC022600F
:102F3000246029C0286027C0206125C027FD2CC03F
:102F4000382F30533A3098F426FF08C08E2D880F62
:102F5000E82EEE0CEE0CE80EE30E15C08F2D880F58
:102F6000F82EFF0CFF0CF80EF30E20620CC08E3210
:102F700021F426FD67C1206406C08C3611F4206858
:102F800002C0883649F4F20193FD859193FF819147
:102F90002F01882309F0BACF982F9554933018F059
:102FA0009052933020F40C5F1F4F39820DC083364E
:102FB00031F0833771F0833509F058C01EC0F80135
:102FC000808189830E5F1F4F540151E0652E712C63
:102FD00012C0F801A080B18026FD03C06FEF7FEF23
:102FE00002C06E2D70E00E5F1F4FC5012C870E943E
:102FF0005C193C012C852F7713C0F801A080B180AB
:1030000026FD03C06FEF7FEF02C06E2D70E00E5FF4
:103010001F4FC5012C870E9451193C012C85206847
:1030200023FF09C01FC080E290E0B6012C870E94F8
:103030006719FA942C858F2D90E06816790698F31D
:1030400011C0F50127FD859127FF81915F0190E077
:10305000B6012C870E9467192C85F110FA94089408
:10306000610871086114710461F7E9C0843611F0D8
:10307000893649F527FF08C0F80160817181828196
:1030800093810C5F1F4F09C0F8016081718188270F
:1030900077FD8095982F0E5F1F4F4FE6B42EB2221A
:1030A00097FF09C090958095709561957F4F8F4FE0
:1030B0009F4FF0E8BF2AA4012AE030E00E94931954
:1030C000782E781843C0853731F43FEEB32EB22204
:1030D0002AE030E023C099EFB92EB2228F3661F09A
:1030E000803720F4883509F0ADC012C0803739F040
:1030F000883709F0A7C005C028E030E00FC020E104
:10310000B22AB4FE02C084E0B82A20E130E006C052
:10311000B4FE02C0E6E0BE2A20E132E0B7FE08C0FD
:10312000F80160817181828193810C5F1F4F07C01C
:10313000F8016081718180E090E00E5F1F4FA40173
:103140000E949319782E7818FFE7BF22B6FE0BC0B5
:103150002EEFB2227E1438F4B4FE07C0B2FC05C0D4
:103160008FEEB82202C0A72C01C0AE2C8B2DB4FE6E
:103170000DC0FE01E70DF11D9081903319F4E9EEC9
:10318000BE2207C0A394B2FE04C002C0867809F034
:10319000A3946B2CB3FC14C0B0FE0FC0AF1410F09E
:1031A000E72C0BC0E72CEF0CEA18AF2C06C080E22E
:1031B00090E0B6010E946719A394AF14C0F304C055
:1031C000AF1410F4FA1801C0FF2464FE0FC080E3AE
:1031D00090E0B6010E94671962FE1DC061FC03C049
:1031E00088E790E00EC088E590E00BC0862D8678D9
:1031F00091F061FE02C08BE201C080E2B7FC8DE27B
:1032000090E0B6010E94671906C080E390E0B60125
:103210000E946719EA947E14C0F37A94F401E70DD2
:10322000F11D808190E0B6010E9467197720A9F70F
:1032300006C080E290E0B6010E946719FA94FF2070
:10324000C1F748CEF60126813781C9012C96E1E10C
:103250000C940E1ADC01CB01FC01E199FECF06C0F3
:10326000FFBBEEBBE09A31960DB20D92415050403B
:10327000B8F70895DC01CB0103C02D910E944519D8
:1032800041505040D0F70895262FE199FECF9FBBC3
:103290008EBB2DBB0FB6F894E29AE19A0FBE019651
:1032A0000895FC010590615070400110D8F7809599
:1032B00090958E0F9F1F0895FC0161507040019002
:1032C0000110D8F7809590958E0F9F1F08950F934A
:1032D0001F93CF93DF938C01EB018B8181FF1BC088
:1032E00082FF0DC02E813F818C819D812817390777
:1032F00064F4E881F9810193F983E88306C0E885E5
:10330000F985802F0995009731F48E819F81019670
:103310009F838E8302C00FEF1FEFC801DF91CF9113
:103320001F910F910895FA01AA27283051F12031F9
:1033300081F1E8946F936E7F6E5F7F4F8F4F9F4F49
:10334000AF4FB1E03ED0B4E03CD0670F781F891F8B
:103350009A1FA11D680F791F8A1F911DA11D6A0F59
:10336000711D811D911DA11D20D009F468943F910C
:103370002AE0269F11243019305D3193DEF6CF010B
:103380000895462F4770405D4193B3E00FD0C9F7D1
:10339000F6CF462F4F70405D4A3318F0495D31FD3E
:1033A0004052419302D0A9F7EACFB4E0A695979591
:1033B000879577956795BA95C9F700976105710567
:1033C00008959B01AC010A2E0694579547953795B1
:1033D0002795BA95C9F7620F731F841F951FA01D0B
:1033E00008952F923F924F925F926F927F928F92A9
:1033F0009F92AF92BF92CF92DF92EF92FF920F9384
:103400001F93CF93DF93CDB7DEB7CA1BDB0B0FB68D
:10341000F894DEBF0FBECDBF09942A88398848884A
:103420005F846E847D848C849B84AA84B984C884E0
:10343000DF80EE80FD800C811B81AA81B981CE0FD7
:10344000D11D0FB6F894DEBF0FBECDBFED010895BC
:04345000F894FFCF1E
:1034540000000003000000008E02230300000000AF
:10346400000200000000B4150000000025322E64A4
:1034740020002A2043414C4942524154494E47209E
:103484002A200043414C2041503D25322E642045E2
:10349400503D25322E642000415A3D25332E6420B0
:1034A400454C3D25332E642025632563004D414E54
:1034B4002041503D25322E642045503D25322E6456
:1034C4002000494E492041503D25322E642045506C
:1034D4003D25322E6420004155544F002538732079
:1034E40025332E642025332E64004445544543542B
:1034F400202020524F544F52532000415A202D2057
:103504004F4B2000415A202D204E4400454C202D85
:0E351400204F4B2000454C202D204E4400003F
:00000001FF
